:100000000C94E4050C942B060C942B060C942B06F4
:100010000C942B060C942B060C942B060C942B069C
:100020000C942B060C942B060C94740D0C942B063C
:100030000C94211C0C942B060C942B060C942B0670
:100040000C942B060C942B060C942B060C942B066C
:100050000C942B060C94C11C0C942B060C942B06B0
:100060000C942B060C942B060C942B060C942B064C
:100070000C942B060C942B060C942B060C942B063C
:100080000C942B060C942B060C942B060C942B062C
:100090000C942B060C942B060C942B060C942B061C
:1000A0000C942B060C942B060C942B066A0E8C0ECB
:1000B0007A0F8C0E7A0FD10EF40E7A0F490F5C0F67
:1000C0006312631290129012EB1227131F151F1563
:1000D0003F131F153A143A14F5141F151F150B156D
:1000E0008080352B787939808080210877060780D9
:1000F0008080201A7A1B168080801E802980808054
:100100008080808080808080808022158019098096
:1001100080801F147B1D0480808023172C050A809B
:100120008080260C00360E808080251876100D8089
:100130008080241C80110B80808027127E370F80E6
:1001400080802A804F7D2880808074305152328098
:1001500080802D137C38338080802E2F5075348022
:10016000253032583A20253038620A000A722F634F
:100170002030313233343536370A005B735D004B43
:100180006579626F6172642073746172742E0A0003
:1001900055534220636F6E666967757265642E0AF7
:1001A000005B575D005B535D005B525D005B445D2F
:1001B000005B435D001203480048004B00420020F2
:1001C000006D006F00640000000E0374002E006DCF
:1001D000002E006B002E0000000403090409028DAC
:1001E00000050100A032090400000103010100091B
:1001F00021110100012240000705810308000A09BE
:100200000401000103010200092111010001224D36
:10021000000705820308000A090402000103000028
:10022000000921110100012236000705830308009F
:100230000A09040300020300000009211101000162
:100240002222000705840320000107050403200083
:10025000010904040001030000000921110100014B
:10026000223900070585031000011201100100006A
:100270000008EDFEFECA04010102000105010906A5
:10028000A101050719E029E7150025019508750169
:10029000810205081901290595057501910295014D
:1002A0007503910105071900297715002501957837
:1002B00075018102C00631FF0974A101097515009D
:1002C00026FF009520750881020976150026FF009B
:1002D000952075089102C005010980A101850216CB
:1002E000010026B7001A01002AB700751095018198
:1002F00000C0050C0901A1018503160100269C021E
:100300001A01002A9C02751095018100C00501099F
:1003100002A1010901A100050919012905150025FE
:10032000019505750181029501750381010501099A
:100330003009311581257F95027508810609381528
:1003400081257F950175088106050C0A3802158103
:10035000257F950175088106C0C005010906A10128
:10036000050719E029E715002501950875018102A7
:100370009501750881010508190129059505750183
:1003800091029501750391010507190029FF1500D8
:1003900026FF00950675088100C00A0025303258F6
:1003A00020006B6579626F6172645F7265706F7255
:1003B000743A20004C45443A20253032580A0064F3
:1003C000656C5F6B65795F6269743A2063616E2763
:1003D000742064656C3A20253032580A00616464E8
:1003E0005F6B65795F6269743A2063616E27742080
:1003F0006164643A20253032580A004F6E65736894
:100400006F743A2074696D656F75740A00646F6E5D
:10041000652E0A00626F6F746D6167696320736394
:10042000616E3A202E2E2E2000290A002575002FFD
:10043000002575005D28002564002000256400204B
:100440000025640020002564007C0025303258001F
:100450006D6F7573656B6579205B62746E7C782057
:1004600079207620685D287265702F61636C293A67
:10047000205B006D6B5F776865656C5F74696D65A7
:100480005F746F5F6D6178203D2025640A006D6B9D
:100490005F776865656C5F6D61785F7370656564D3
:1004A000203D2025640A006D6B5F74696D655F7483
:1004B0006F5F6D6178203D2025640A006D6B5F6D74
:1004C00061785F7370656564203D2025640A006D66
:1004D0006B5F696E74657276616C203D2025640ADD
:1004E000006D6B5F64656C6179203D2025640A00B6
:1004F0006D6B5F776865656C5F74696D655F746F60
:100500005F6D6178203D2025640A006D6B5F776820
:1005100065656C5F6D61785F7370656564203D2013
:1005200025640A006D6B5F74696D655F746F5F6D44
:100530006178203D2025640A006D6B5F6D61785FF6
:100540007370656564203D2025640A006D6B5F69EA
:100550006E74657276616C203D2025640A006D6BB7
:100560005F64656C6179203D2025640A000A0025DE
:100570007500363A20776865656C5F74696D655FF4
:10058000746F5F6D61783A20000A00257500353A76
:1005900020776865656C5F6D61785F737065656411
:1005A0003A20000A00257500343A2074696D655FB1
:1005B000746F5F6D61783A20000A00257500333A48
:1005C000206D61785F73706565643A20000A0025CC
:1005D0007500323A20696E74657276616C286D73AD
:1005E000293A20000A00257500313A2064656C61C3
:1005F00079282A31306D73293A20000A092D2056B6
:10060000616C756573202D0A004D3E004D25643EDA
:1006100020003F007365742064656661756C740A20
:1006200000433E200077686572652064656C7461E4
:100630003A20637572736F723D25642C207768656C
:10064000656C3D25640A53656520687474703A2FA3
:100650002F656E2E77696B6970656469612E6F72A4
:10066000672F77696B692F4D6F7573655F6B657960
:10067000730A000A092D204D6F7573656B6579202B
:100680002D0A4553432F713A09717569740A313A3D
:100690000964656C6179282A31306D73290A323A10
:1006A00009696E74657276616C286D73290A333A34
:1006B000096D61785F73706565640A343A0974691D
:1006C0006D655F746F5F6D61780A353A09776865AB
:1006D000656C5F6D61785F73706565640A363A09B1
:1006E000776865656C5F74696D655F746F5F6D6178
:1006F000780A0A703A097072696E742076616C75B6
:1007000065730A643A097365742064656661756C83
:1007100074730A75703A092B310A646F776E3A095F
:100720002D310A706775703A092B31300A70676491
:100730006F776E3A092D31300A0A7370656564204F
:100740003D2064656C7461202A206D61785F737050
:10075000656564202A2028726570656174202F20E9
:1007600074696D655F746F5F6D6178290A003F0081
:100770004D3E2000433E20004C25640A000A092D0E
:1007800020436F6E736F6C65202D0A4553432F71A4
:100790003A09717569740A6D3A096D6F7573656B05
:1007A00065790A000A092D204D61676963202D0AC9
:1007B000643A0964656275670A783A096465627526
:1007C00067206D61747269780A6B3A0964656275B5
:1007D00067206B6579626F6172640A6D3A096465BE
:1007E000627567206D6F7573650A763A0976657272
:1007F00073696F6E0A733A097374617475730A636F
:100800003A09636F6E736F6C65206D6F64650A30B3
:100810002D343A096C61796572302D3428463130B7
:100820002D4634290A506175733A09626F6F746CF2
:100830006F616465720A653A09656570726F6D0A69
:100840006E3A094E4B524F0A000A002575002E6E73
:100850006B726F3A20000A002575002E7377617065
:100860005F6261636B736C6173685F6261636B731A
:10087000706163653A20000A002575002E73776168
:10088000705F67726176655F6573633A20000A0086
:100890002575002E6E6F5F6775693A20000A002586
:1008A00075002E737761705F72616C745F7267752B
:1008B000693A20000A002575002E737761705F6C1D
:1008C000616C745F6C6775693A20000A00257500D9
:1008D0002E636170736C6F636B5F746F5F636F6EB9
:1008E00074726F6C3A20000A002575002E737761D0
:1008F000705F636F6E74726F6C5F636170736C6F47
:10090000636B3A20000A0025303258006B65796D20
:1009100061705F636F6E6669672E7261773A20005F
:100920000A002575002E6D6F7573653A20000A0068
:100930002575002E6B6579626F6172643A20000A3A
:10094000002575002E6D61747269783A20000A00E6
:100950002575002E656E61626C653A20000A0025DF
:100960003032580064656275675F636F6E666967F1
:100970002E7261773A20000A002575006465666171
:10098000756C745F6C617965723A20003F004E4B64
:10099000524F3A206F66660A004E4B524F3A206F14
:1009A0006E0A0074696D65725F7265616433322826
:1009B000293A202530346C580A006B6579626F61E2
:1009C00072645F6E6B726F3A2025580A006B65790E
:1009D000626F6172645F69646C653A2025580A0031
:1009E0006B6579626F6172645F70726F746F636F51
:1009F0006C3A2025580A00686F73745F6B657962E2
:100A00006F6172645F6C65647328293A2025580A07
:100A1000000A092D20537461747573202D0A004754
:100A200043433A20342E392E32204156522D4C4920
:100A300042433A20312E382E3073766E2041565282
:100A40005F415243483A20617672350A004F505454
:100A5000494F4E533A204C55464120424F4F544D3A
:100A600041474943204D4F5553454B455920455823
:100A70005452414B455920434F4E534F4C45204310
:100A80004F4D4D414E44204E4B524F204B45594DFA
:100A900041505F53454354494F4E20343039360A54
:100AA000004255494C443A20363233653034652093
:100AB0002831333A35353A313420417567203236A2
:100AC0002032303136290A005649443A20307846DF
:100AD00045454428742E6D2E6B2E29205049443AEA
:100AE000203078434146452848484B42206D6F648A
:100AF00029205645523A203078303130340A0044AB
:100B00004553433A20742E6D2E6B2E206B6579620F
:100B10006F617264206669726D7761726520666FBD
:100B2000722048484B42206D6F640A000A092D204C
:100B300056657273696F6E202D0A000A6D6F7573AA
:100B4000653A206F66660A000A6D6F7573653A2014
:100B50006F6E0A000A6B6579626F6172643A206F8A
:100B600066660A000A6B6579626F6172643A206F8B
:100B70006E0A000A6D61747269783A206F66660ABF
:100B8000000A6D61747269783A206F6E0A000A6417
:100B9000656275673A206F6E0A000A646562756760
:100BA0003A206F66660A000A0A626F6F746C6F61A2
:100BB0006465722E2E2E2000433E20006565636F13
:100BC0006E6669673A0A000011241FBECFEFDAE0B3
:100BD000DEBFCDBF04B603FE27C080910202909114
:100BE0000302A0910402B09105028730904BA74008
:100BF000B04BD1F410920202109203021092040240
:100C00001092050214BE84B7877F84BF0FB6F89494
:100C1000A8958091600088618093600010926000C8
:100C20000FBEE0E0F8E3099511E0A0E0B1E0EAE2F0
:100C3000F1E502C005900D92A833B107D9F722E083
:100C4000A8E3B1E001C01D92A230B207E1F70E9413
:100C50009C0A0C9493280C940000FF93EF93E0916E
:100C60003801F0913901309709F00995EF91FF9122
:100C70000895FC018591803011F0EFDFFBCF0895DE
:100C8000FF27E0E230E247FF0CC0419597FF09C023
:100C9000EDE26095709580959095611D711D811DA7
:100CA000911D27FF02C0219530E350E2AA27660F6D
:100CB000771F881F991FAA1FA41710F0A41B639504
:100CC0005A95A9F7AA3008F0A95FA05DAF93F395F4
:100CD000611571058105910541F7ED3211F4EF932E
:100CE000F395F21718F43F93F395FBCF8F91B5DF8F
:100CF000FA95E1F70895E991F9918591803021F015
:100D0000853219F0AADFF9CF089520E0E8945591D3
:100D10005532C1F3503311F4689455915A3348F465
:100D2000505390F3220F022E220F220F200D250F79
:100D3000F4CF0EF4219589919991533619F35337D5
:100D400029F1533559F1BC0188279927E8945C367D
:100D500021F48991999168945591543639F446EF6C
:100D60007EF077FF0DC08FEF9FEF0AC055374AE046
:100D700039F0583540E121F0523642E009F008954B
:100D8000FF93EF937DDFEF91FF91B7CFFF93EF9349
:100D9000FC0181918030B9F360DFFBCFFF93EF93CB
:100DA00068DFF1CFDF93CF93CDB7DEB72596A3DF12
:100DB000CF91DF9108958FEF84B980E485B957987A
:100DC0005F9A87B1806C87B988B1806C88B92E9A98
:100DD0002F98EAE4F1E080E18E0F11928E13FDCF9F
:100DE000EAE3F1E080E18E0F11928E13FDCF8AE4E9
:100DF00091E090935D0180935C018AE391E0909390
:100E00005B0180935A010895EF92FF920F931F9315
:100E1000CF93DF9380915A0190915B0120915C0107
:100E200030915D0130935B0120935A0190935D01F5
:100E300080935C01C0E0D0E001E010E080E090E051
:100E4000FC2FF770EC2FE87025B1207C2F2BAC0124
:100E500033E0440F551F3A95E1F7242B25B928B10B
:100E60002F73EE2311F0206401C0206828B92AE115
:100E70002A95F1F700C0A0915A01B0915B01AC0F27
:100E8000BD1F2C9130E0082E02C0359527950A949D
:100E9000E2F720FD2F9AA5E3AA95F1F70000F6B43A
:100EA0002E98BAE1BA95F1F700C040915C015091DB
:100EB0005D01BA016C0F7D1F4F9B0BC09801082E7E
:100EC00001C0220F0A94EAF72095DB013C9123230D
:100ED00009C0DB01EC909801082E01C0220F0A9492
:100EE000EAF72E292C9326B56F2D70E02F1518F0F8
:100EF00026B530E004C026B530E021503F4F261B18
:100F0000370B2630310558F0A0915A01B0915B01A2
:100F1000AC0FBD1F2C91DA01AC0FBD1F2C93BAE1B1
:100F2000BA95F1F700C02F982E9A20EA2A95F1F78A
:100F300001968830910509F087CFA0915C01B091AE
:100F40005D01AC0FBD1FE0915A01F0915B01EC0F08
:100F5000FD1F9C918081981751F00E945F1C609347
:100F60005E0170935F01809360019093610121960F
:100F7000C031D10509F062CF8091F801853021F0B0
:100F80008091F801811111C060915E0170915F0143
:100F900080916001909161010E94951C61317742BE
:100FA0008105910510F00E94E21B81E0DF91CF9155
:100FB0001F910F91FF90EF90089520915C01309167
:100FC0005D01F901E80FF11D808108950F931F93D2
:100FD000CF93DF938CE691E00E943906C0E0D0E029
:100FE00000E611E0E0915C01F0915D01EC0FFD1F66
:100FF00080810E94B71B1F928F93DF93CF931F9323
:101000000F930E94D20621960F900F900F900F9091
:101010000F900F90C031D10529F7DF91CF911F912B
:101020000F91089508950895569A81FF02C05E9A1F
:1010300008955E9808958091750108959FB7F8947A
:10104000109264019FBF9091F801943009F057C04D
:101050009091E9009F703091EC00232F217030FDBA
:1010600020E8922B24E02093E9002091EB0020FF60
:1010700043C02091EE0027FF3FC020916201222350
:1010800021F02091E80025FF37C01092620126E090
:101090003091E80035FD15C03091F801343061F52C
:1010A0003091EB0035FD28C0215021F481E0809380
:1010B000620122C0EFE9FFE03197F1F700C00000C4
:1010C000E7CF8093F1008091E80085FD0AC0809110
:1010D000E80080FFFCCF8091E8008E778093E800E5
:1010E00006C08FB7F89421E0209364018FBF9F70F2
:1010F0009093E90080E008959F709093E9008FEF4E
:101100000895CF93DF9300D01F92CDB7DEB79C0137
:101110008091F801843019F593E099833B832A8309
:101120009093E9008FEF9091E800815095FD06C003
:1011300095ED9A95F1F700008111F5CF8091E800C7
:1011400085FF0DC040E050E063E070E0CE01019605
:101150000E94620B8091E8008E778093E8000F90E8
:101160000F900F90DF91CF910895CF93DF9300D030
:101170001F92CDB7DEB72091F801243021F522E08F
:1011800029839B838A8383E08093E9008FEF90918A
:10119000E800815095FD06C095ED9A95F1F70000A5
:1011A0008111F5CF8091E80085FF0DC040E050E04F
:1011B00063E070E0CE0101960E94620B8091E8002E
:1011C0008E778093E8000F900F900F90DF91CF9172
:1011D00008952091F8012430F1F422E02093E900F1
:1011E0002FEF3091E800215035FD06C035ED3A95DE
:1011F000F1F700002111F5CF2091E80025FF0BC089
:1012000040E050E065E070E00E94620B8091E800F1
:101210008E778093E8000895CF93DF932091F801B3
:10122000243009F048C0EC0180910A018823E1F0E4
:1012300080910B018823C1F085E08093E9008FEF56
:101240009091E800815095FD06C095E19A95F1F7DF
:1012500000008111F5CF8091E80085FF2CC040E0AF
:1012600050E060E170E017C081E08093E9008FEF0B
:101270009091E800815095FD06C095ED9A95F1F7A3
:1012800000008111F5CF8091E80085FF14C040E097
:1012900050E068E070E0CE010E94620B8091E800AF
:1012A0008E778093E80080E1FE01A5E6B1E0019031
:1012B0000D928A95E1F7DF91CF91089581EB91E04E
:1012C0000E9439068091F701811109C00E94F90C32
:1012D0000E94560D8091E20084608093E2000895A0
:1012E0008DEA91E00E9439061092F701089589EA8B
:1012F00091E00C943906209163012F5F822F62E305
:101300000E942828992319F02093630108951092D0
:10131000630180916401882371F18091F801843028
:1013200041F58091E9008F702091EC00922F91702F
:1013300020FD90E8892B94E09093E9009091EB00D8
:1013400090FF14C09091EE0097FF10C09091E800BC
:1013500095FF03C01092F100F9CF9091E80090FF43
:1013600005C09091E8009E779093E8008F7080937D
:10137000E90010926401089542E061EC81E00E946E
:10138000730C42E061EC82E00E94730C42E061EC7D
:1013900083E00E94730C42E261EC84E00E94730CD3
:1013A00042E161EC85E00C94730C8091FA0183308A
:1013B00009F455C030F4813071F0823009F48EC0E8
:1013C00008958A3009F47AC08B3009F460C08930FE
:1013D00009F09CC020C08091F901813A09F096C0C3
:1013E0008091E800877F8093E8008091FD019091D3
:1013F000FE01892B21F460E185E691E003C060E005
:1014000080E090E070E00E94AF0B8091E8008B7765
:101410008093E80008958091F901813209F076C047
:101420008091FD019091FE01009719F0049709F059
:101430006DC08091E800877F8093E8008091E8008C
:1014400082FD05C08091F8018111F8CF5FC08091C5
:10145000F100809375018091E8008B7753C08091F3
:10146000F901813A09F052C08091FD019091FE018D
:10147000892B09F04BC08091E800877F8093E800BA
:101480008091E80080FFFCCF80910A0136C08091F6
:10149000F9018132D9F58091FD019091FE01892BEE
:1014A000A9F58091E800877F8093E8000E94A80C4E
:1014B0008091FB0180930A010C9440158091F90101
:1014C000813221F58091E800877F8093E8000E94B7
:1014D000A80C8091FC018093760108958091F90118
:1014E000813AA1F48091E800877F8093E8008091A1
:1014F000E80080FFFCCF809176018093F10080911D
:10150000E8008E778093E8000C94A80C0895089565
:101510000895089585EA91E00E9439060C94890A9D
:101520000E94E21B8091F601882329F00E940B1C87
:1015300081110C944C0B089584B7877F84BF0FB63C
:10154000F894A89580916000886180936000109263
:1015500060000FBE90E080E80FB6F89480936100C1
:10156000909361000FBE0E94870A0E943F100E9464
:10157000F90C0E94560D8091E20084608093E20095
:101580008EE198E00E94B21B78948091F80184303B
:1015900019F00E94920FF9CF80E991E00E9439067C
:1015A0000E94411080E091E00E94AD0F8FE791E032
:1015B0000E9439060E94880A8091F801853039F42A
:1015C0008BE791E00E9439060E94900AF5CF0E94B5
:1015D00047100E94920FF0CF0C941F1C81EA91E0FB
:1015E0000E9439060C94EC0A292F33272330310549
:1015F000C9F064F42130310581F02230310509F061
:1016000043C08DE890E02DED31E042C0213231053C
:10161000F1F02232310541F137C082E190E02AE653
:1016200032E036C099278130910541F08230910532
:1016300041F0892B49F5E9EDF1E005C0E9ECF1E075
:1016400002C0E5EBF1E0849190E09F0121C065309C
:10165000D8F4E62FF0E0EE0FFF1FED5DFE4F208186
:10166000318189E090E014C0653070F470E0FB01D6
:10167000EE0FFF1FE75EFE4F20813181FB01EC5E24
:10168000FE4F808190E004C080E090E020E030E0F8
:10169000FA0131832083089580E189BD82E189BD0B
:1016A00009B400FEFDCF8091D8008F7D8093D800D3
:1016B0008091E00082608093E0008091E00081FDF5
:1016C000FCCF0895CF92DF92EF92FF920F931F937A
:1016D000CF93DF93EC018B017A010E94C70C81113B
:1016E00035C0E114F10439F0F70180819181081BC4
:1016F000190BC80FD91FC12CD12C0115110529F1C7
:101700008091E80085FD18C08091E8008E77809375
:10171000E8000E94920FE114F10449F0F701808182
:101720009181C80ED91ED182C08285E00FC00E946F
:10173000C70C882311F30AC089918093F1000150EE
:101740001109FFEFCF1ADF0AD8CF80E0DF91CF91E8
:101750001F910F91FF90EF90DF90CF90089520910F
:10176000FF01309100022617370748F06115710517
:1017700039F42091E8002E772093E80001C0B901E8
:1017800040E061157105A9F12091F801222309F4C7
:1017900043C0253009F442C02091E80023FD40C039
:1017A0002091E80022FD32C02091E80020FFE9CF1F
:1017B0004091F3002091F20030E0342BFC01CF0186
:1017C0006115710559F02830310540F481918093FD
:1017D000F100615071092F5F3F4FF1CF41E0283098
:1017E000310509F040E02091E8002E772093E800D1
:1017F000C8CF4111C9CF0AC08091F801882361F098
:10180000853061F08091E80083FD0AC08091E80096
:1018100082FFF2CF80E0089582E0089583E008958A
:1018200081E008952091FF013091000226173707CB
:1018300048F06115710539F42091E8002E77209366
:10184000E80001C0B901FC0120E06115710591F1CA
:101850008091F801882309F440C0853009F43FC025
:101860008091E80083FD3DC08091E80082FD2FC09B
:101870008091E80080FFE9CF2091F3008091F20091
:1018800090E0922B6115710559F08830910540F474
:1018900024912093F1003196615071090196F2CFA5
:1018A00021E0089709F020E08091E8008E7780938E
:1018B000E800CBCF2111CCCF0AC08091F80188235A
:1018C00061F0853061F08091E80083FD0AC080916D
:1018D000E80082FFF2CF80E0089582E0089583E07F
:1018E000089581E00895982F973058F59093E90076
:1018F000981739F07091EC002091ED005091F000B4
:1019000003C0242F762F50E021FF19C03091EB0047
:101910003E7F3093EB003091ED003D7F3093ED0042
:101920003091EB0031603093EB007093EC0020932A
:10193000ED005093F0002091EE0027FF07C09F5F5D
:10194000D3CF8F708093E90081E0089580E00895FF
:101950008091F90187FF11C08091E80082FD05C0E8
:101960008091F8018111F8CF11C08091E8008B7748
:101970000BC08091F801882349F08091E80080FF36
:10198000F8CF8091E8008E778093E8000895209149
:10199000E4003091E50095E64091EC00842F8170E1
:1019A00040FF22C08091E80080FD1CC08091F801BA
:1019B000882391F0853091F08091EB0085FD10C077
:1019C0004091E4005091E5004217530729F39A0132
:1019D000915011F784E0089582E0089583E008951E
:1019E00081E0089580E008954091E80042FFDECF55
:1019F00008950E94670D0E946F0DE0EEF0E0808177
:101A000081608083E8EDF0E080818F77808319BC6E
:101A1000A7EDB0E08C918E7F8C9380818F7E808348
:101A20001092F70108950F931F93CF93DF930E94B5
:101A3000670D0E946F0DC8EDD0E088818F77888395
:101A400088818068888388818F7D888319BC109203
:101A5000F8011092F4011092F6011092F50100EED7
:101A600010E0F80180818B7F80838881816088838A
:101A700042E060E080E00E94730CE1EEF0E08081E3
:101A80008E7F8083E2EEF0E08081816080838081C0
:101A900088608083F80180818E7F80838881806167
:101AA0008883DF91CF911F910F910895E8EDF0E0C9
:101AB00080818F7E8083E7EDF0E08081816080838C
:101AC00084E082BF81E08093F7010C94130DE8ED70
:101AD000F0E080818E7F80831092E2000895109262
:101AE000DA001092E10008951F920F920FB60F9244
:101AF00011242F933F934F935F936F937F938F9313
:101B00009F93AF93BF93EF93FF938091E10082FF88
:101B10000BC08091E20082FF07C08091E1008B7FC3
:101B20008093E1000E947B098091DA0080FF1FC052
:101B30008091D80080FF1BC08091DA008E7F809357
:101B4000DA008091D90080FF0DC080E189BD82E17B
:101B500089BD09B400FEFDCF81E08093F8010E94A9
:101B60005E0905C019BC1092F8010E9470098091AD
:101B7000E10080FF19C08091E20080FF15C08091D4
:101B8000E2008E7F8093E2008091E200806180938A
:101B9000E2008091D80080628093D80019BC85E073
:101BA0008093F8010E948A0A8091E10084FF30C08E
:101BB0008091E20084FF2CC080E189BD82E189BD73
:101BC00009B400FEFDCF8091D8008F7D8093D800AE
:101BD0008091E1008F7E8093E1008091E2008F7E12
:101BE0008093E2008091E20081608093E200809126
:101BF000F401882311F084E007C08091E30087FDA1
:101C000002C081E001C083E08093F8010E94EE0AE7
:101C10008091E10083FF24C08091E20083FF20C017
:101C20008091E100877F8093E10082E08093F8015A
:101C30001092F4018091E1008E7F8093E100809109
:101C4000E2008E7F8093E2008091E20080618093C9
:101C5000E20042E060E080E00E94730C0E9477099D
:101C6000FF91EF91BF91AF919F918F917F916F9174
:101C70005F914F913F912F910F900FBE0F901F904A
:101C800018951F93CF93DF93CDB7DEB7AA970FB602
:101C9000F894DEBF0FBECDBFE9EFF1E088E08E0F14
:101CA0009091F10091938E13FBCF0E94D509809102
:101CB000E80083FF1FC18091F9019091FA01492F3B
:101CC00050E04A30510508F015C1FA01EA5AFF4FB9
:101CD0000C944828803881F0823809F00BC180913B
:101CE000FD018F708093E9008091EB0085FB8827D0
:101CF00080F91092E90006C08091F5019091F601FB
:101D0000911182609091E800977F9093E800809312
:101D1000F1001092F100C8C0282F2D7F09F0EAC011
:101D2000882319F0823061F0E5C08091FB01813099
:101D300009F0E0C0933009F080E08093F6012BC0F9
:101D40008091FB01811127C08091FD018F7009F402
:101D5000D1C08093E9002091EB0020FF1CC093309C
:101D600021F48091EB00806214C09091EB009061AF
:101D70009093EB0021E030E0A90102C0440F551F11
:101D80008A95E2F74093EA001092EA008091EB0016
:101D900088608093EB001092E9008091E800877FD3
:101DA00086C08111A7C01091FB011F778091E300CD
:101DB0008078812B8093E3008091E800877F809377
:101DC000E8000E94A80C8091E80080FFFCCF809181
:101DD000E30080688093E300111102C082E001C03B
:101DE00083E08093F80186C08058823008F082C07A
:101DF0008091FB019091FC018C3D53E0950779F5B2
:101E000083E08A838AE289834FB7F894DE011396D0
:101E100020E03EE051E2E32FF0E050935700E491E0
:101E200020FF03C0E295EF703F5FEF708E2F90E0D0
:101E3000EA3010F0C79601C0C0968D939D932F5F36
:101E4000243149F74FBF8091E800877F8093E800F5
:101E50006AE270E0CE0101960E94AF0B14C0AE01A1
:101E60004F5F5F4F6091FD010E94F40ABC01892B16
:101E700009F440C09091E800977F9093E800898131
:101E80009A810E94120C8091E8008B778093E80081
:101E900031C0803879F58091E800877F8093E80031
:101EA0008091F4018093F1008091E8008E77809317
:101EB000E8000E94A80C1EC081111CC09091FB017B
:101EC0009230C0F48091E800877F8093E80090937F
:101ED000F4010E94A80C8091F401811106C0809148
:101EE000E30087FD02C081E001C084E08093F80137
:101EF0000E94BC098091E80083FF0AC08091E8003D
:101F0000877F8093E8008091EB0080628093EB00F4
:101F1000AA960FB6F894DEBF0FBECDBFDF91CF916A
:101F20001F910895CF938091F8018823A1F0C0916B
:101F3000E900CF709091EC00892F817090FD80E8CE
:101F4000C82B1092E9008091E80083FD0E94410EA9
:101F5000CF70C093E900CF91089590937C01809356
:101F60007B010895E0917B01F0917C01309721F095
:101F70000190F081E02D099480E00895EF92FF92A6
:101F80000F931F93CF93DF93E0917B01F0917C013E
:101F90003097B1F18C010280F381E02D0995809199
:101FA000E30182FF2DC080FF04C082EA93E00E941B
:101FB0003906E80110E18CE9E82E83E0F82E8091E3
:101FC000E30180FF0BC088811F928F93FF92EF92F5
:101FD0000E94D2060F900F900F900F9011502196F3
:101FE0001111EDCF8091E30180FF0AC08AE993E0EF
:101FF000DF91CF911F910F91FF90EF900C943906D4
:10200000DF91CF911F910F91FF90EF900895E09194
:102010007B01F0917C01309721F00480F581E02D67
:10202000099408952091790130917A0182179307DC
:1020300071F090937A0180937901E0917B01F091A6
:102040007C01309721F00680F781E02D09940895F6
:1020500020917701309178018217930771F0909366
:10206000780180937701E0917B01F0917C013097BA
:1020700021F00084F185E02D0994089508950C94D1
:102080003E100E944A1C0E94DB060C94981DCF92C1
:10209000DF92EF92FF920F931F93CF93DF9300D0C5
:1020A00000D000D0CDB7DEB70E9404078EE7C82E5F
:1020B00081E0D82E00E010E0E02E802F0E94DD07A6
:1020C000F60141916F01F42EF826B1F40F5F1F4F16
:1020D0000031110589F78FEF89838A831B820E9463
:1020E000531C8160782F9D838C8349815A816B8139
:1020F0008D810E94061147C09091E30191FF04C0B9
:102100008E830E94E6078E8120E030E04F2D50E064
:10211000922FBA01022E02C0759567950A94E2F7D4
:1021200060FF2BC02983EA8221E030E0690102C010
:10213000CC0CDD1C9A95E2F790E08C219D21892B37
:1021400009F420E02B830E94531C8160782F9D832B
:102150008C8349815A816B818D810E94061149814E
:102160005A816B817C818D810E94CE1BF801E258DF
:10217000FE4F8081C826C08206C02F5F3F4F2830A7
:10218000310531F6A3CF0E94CD1B0E942221109170
:102190007D010E94B20F181741F10E94B20F809387
:1021A0007D019091E30192FF0EC090FF0CC01F9241
:1021B0008F9384EB93E09F938F930E94D2060F90AE
:1021C0000F900F900F9080917D0126960FB6F89496
:1021D000DEBF0FBECDBFDF91CF911F910F91FF905A
:1021E000EF90DF90CF900C94DF1B26960FB6F894FB
:1021F000DEBF0FBECDBFDF91CF911F910F91FF903A
:10220000EF90DF90CF9008950C941408CF93DF9354
:10221000CDB7DEB72B970FB6F894DEBF0FBECDBF9C
:10222000942F4F83252F588769877A878B874A8514
:102230005B85452B21F02F3F09F59F3FF9F4DE0127
:10224000119686E0FD0111928A95E9F785E0FE017D
:10225000379601900D928A95E1F749815A816B81F9
:102260007C818D819E810E94E3172B960FB6F89496
:10227000DEBF0FBECDBFDF91CF9108954F8158854E
:1022800069857A858B850E94CE1BD9CFCF93882311
:1022900009F4A4C0C82F8CEF8C0F813A48F48C2F1E
:1022A0000E94A22581119AC08C2F0E946E1A0CC028
:1022B00080E28C0F883058F4C77081E001C0880F2D
:1022C000CA95EAF70E94191BCF910C945D1B8BE510
:1022D0008C0F833078F4C53A29F0C63A31F083E8A0
:1022E00090E005C081E890E002C082E890E0CF91E4
:1022F0000C94121088E58C0F853108F06FC0C83A35
:1023000061F1C93A69F1CA3A71F1CB3A79F1CC3A43
:1023100081F1CD3A89F1CE3A91F1CF3A99F1C13BB1
:10232000A1F1C03BA9F1C23BB1F1C33BB9F1C43B40
:10233000C1F1C53BC9F1C63BD1F1C73BD9F1C83B9F
:10234000E1F1C93BE9F1CA3BF1F1CB3BF9F1CC3BFF
:1023500009F43FC080E090E03EC082EE90E03BC0D8
:1023600089EE90E038C08AEE90E035C085EB90E0D1
:1023700032C086EB90E02FC083EB90E02CC084EB62
:1023800090E029C087EB90E026C08CEC90E023C061
:102390008DEC90E020C083E891E01DC08AE891E0D8
:1023A0001AC082E991E017C084E991E014C081E28B
:1023B00092E011C083E292E00EC084E292E00BC092
:1023C00085E292E008C086E292E005C087E292E0F2
:1023D00002C08AE292E0CF910C942810CF91089528
:1023E000882329F19CEF980F913A18F40E94C11AA2
:1023F0000DC090E2980F983058F4877091E001C0BA
:10240000990F8A95EAF7892F0E941F1B0C945D1B78
:102410009BE5980F933020F480E090E00C9412102C
:10242000885A853120F480E090E00C9428100895BB
:10243000882321F00E94191B0C945D1B08958823AA
:1024400021F00E941F1B0C945D1B0895CF92DF9218
:10245000EF92FF920F931F93CF93DF9300D000D0A2
:1024600000D0CDB7DEB725E0FC01DE01119601906A
:102470000D922A95E1F7FC0140813181F28025819E
:1024800022952F7063817481672B09F4D8C23F3F76
:1024900019F44F3F09F4D3C26C0149833A8389810F
:1024A0009A812E830E942D1A182F092F0E942C1A10
:1024B0000E943C19E02FE295EF70F0E0E05AFF4FE8
:1024C0002E810C944828802F807F902F9F70092F99
:1024D000882311F00295007FFF2049F0002309F4C2
:1024E0005FC2802F0E942C1B0E945D1B59C2812F4E
:1024F0000E94F011002309F4A2C2802F0E94321B17
:1025000026960FB6F894DEBF0FBECDBFDF91CF91F8
:102510001F910F91FF90EF90DF90CF900C945D1B77
:10252000802F807F902F9F70092F803211F00295AD
:10253000007F112319F0113001F129C0FF20A9F00B
:10254000802F222349F1213039F526960FB6F894D1
:10255000DEBF0FBECDBFDF91CF911F910F91FF90D6
:10256000EF90DF90CF900C943C1B222319F0213088
:1025700009F465C20E94451B2CC0FF20E9F02630FB
:1025800008F05DC20E94161B802329F022C0FF20A4
:10259000F1F0211115C0802F26960FB6F894DEBFFA
:1025A0000FBECDBFDF91CF911F910F91FF90EF90A4
:1025B000DF90CF900C941812253008F040C209C06B
:1025C000F601858180FFECC18F708583E4CF2111F6
:1025D000FBC1802F69C1202F26952695237030E0FE
:1025E0002115310521F021303105C9F028C2FF2025
:1025F00021F0812F902F937002C080E090E026960A
:102600000FB6F894DEBF0FBECDBFDF91CF911F9103
:102610000F91FF90EF90DF90CF900C941210FF205D
:1026200021F0812F902F937002C080E090E02696D9
:102630000FB6F894DEBF0FBECDBFDF91CF911F91D3
:102640000F91FF90EF90DF90CF900C942810812F86
:10265000FF2019F00E94A81F02C00E941020269699
:102660000FB6F894DEBF0FBECDBFDF91CF911F91A3
:102670000F91FF90EF90DF90CF900C949520802FDA
:10268000837009F078C0F110DAC1812F82958695A8
:102690008770880F880F912F9F70C92ED12CE12C45
:1026A000F12C082E04C0CC0CDD1CEE1CFF1C0A947F
:1026B000D2F714FF12C04FE050E060E070E004C0B9
:1026C000440F551F661F771F8A95D2F7CB01BA01B9
:1026D000609570958095909503C060E070E0CB01A7
:1026E000202F269526952370422F50E04230510529
:1026F000D1F04330510559F16C297D298E299F294C
:102700004130510541F126960FB6F894DEBF0FBE59
:10271000CDBFDF91CF911F910F91FF90EF90DF9090
:10272000CF900C9451196C297D298E299F292696CA
:102730000FB6F894DEBF0FBECDBFDF91CF911F91D2
:102740000F91FF90EF90DF90CF900C9463190E944F
:102750005119C701B60126960FB6F894DEBF0FBE19
:10276000CDBFDF91CF911F910F91FF90EF90DF9040
:10277000CF900C943F19FF2019F0802F817001C079
:102780008695882309F45BC1812F82958695877091
:10279000880F880F912F9F70C92ED12CE12CF12C1E
:1027A000082E04C0CC0CDD1CEE1CFF1C0A94D2F7D2
:1027B00014FF12C04FE050E060E070E004C0440F2E
:1027C000551F661F771F8A95D2F7CB01BA01609516
:1027D00070958095909503C060E070E0CB01202F4C
:1027E000269526952370422F50E042305105D1F0B6
:1027F0004330510559F16C297D298E299F2941309B
:10280000510541F126960FB6F894DEBF0FBECDBF3D
:10281000DF91CF911F910F91FF90EF90DF90CF90BC
:102820000C94081A6C297D298E299F2926960FB6AB
:10283000F894DEBF0FBECDBFDF91CF911F910F91F6
:10284000FF90EF90DF90CF900C941A1A0E94081A14
:10285000C701B60126960FB6F894DEBF0FBECDBFF6
:10286000DF91CF911F910F91FF90EF90DF90CF906C
:102870000C94F619103F41F118F4103E48F48BC047
:10288000123F09F450C0D8F1133F09F460C083C06F
:102890001F70802F8F71FF2021F00E948F19812FD0
:1028A0007BCE0E94B019812F26960FB6F894DEBF1A
:1028B0000FBECDBFDF91CF911F910F91FF90EF9091
:1028C000DF90CF900C941F12FF20A9F0253008F064
:1028D000B6C0802F8F7126960FB6F894DEBF0FBE5C
:1028E000CDBFDF91CF911F910F91FF90EF90DF90BF
:1028F000CF900C94D519263008F0A1C0EACFFF2064
:10290000A1F0802F8F7126960FB6F894DEBF0FBE10
:10291000CDBFDF91CF911F910F91FF90EF90DF908E
:10292000CF900C948F19FF2061F3802F8F71269622
:102930000FB6F894DEBF0FBECDBFDF91CF911F91D0
:102940000F91FF90EF90DF90CF900C94B019FF2083
:1029500091F0802F8F7126960FB6F894DEBF0FBED0
:10296000CDBFDF91CF911F910F91FF90EF90DF903E
:10297000CF900C947A1926960FB6F894DEBF0FBE4E
:10298000CDBFDF91CF911F910F91FF90EF90DF901E
:10299000CF900C947519FF20A1F0222309F4B1CF38
:1029A000812F26960FB6F894DEBF0FBECDBFDF9104
:1029B000CF911F910F91FF90EF90DF90CF900C94EB
:1029C0004611222309F4B1CF812F26960FB6F89431
:1029D000DEBF0FBECDBFDF91CF911F910F91FF9052
:1029E000EF90DF90CF900C94F011402F4F70612F3B
:1029F000C6010E94421D26960FB6F894DEBF0FBE98
:102A0000CDBFDF91CF911F910F91FF90EF90DF909D
:102A1000CF900C948718402F4F70612FC6012696D7
:102A20000FB6F894DEBF0FBECDBFDF91CF911F91DF
:102A30000F91FF90EF90DF90CF900C94451D26965C
:102A40000FB6F894DEBF0FBECDBFDF91CF911F91BF
:102A50000F91FF90EF90DF90CF9008950E94391B67
:102A60000E94081B0E945D1B0E94C7210E949520A6
:102A700080E090E00E94121080E090E00C9428101A
:102A80000E94291B0C942E150E942D1A292F229585
:102A90002F7030E02C3031054CF42A3031056CF4C5
:102AA000225031092230310588F407C02C3031051D
:102AB00049F02F30310531F009C0803E48F0803FA9
:102AC00029F406C093FB882780F9089580E00895D3
:102AD00081E00895CF93DF9300D000D01F92CDB74F
:102AE000DEB70F900F900F900F900F90DF91CF9166
:102AF0000895CF93DF9300D000D000D0CDB7DEB7DC
:102B000026960FB6F894DEBF0FBECDBFDF91CF91F2
:102B100008951F93CF93DF93C0918E0116E08091AB
:102B20008F01C81799F0D0E01C9FF0011D9FF00D98
:102B30001124E057FE4F408151816281738184816D
:102B400095810E9479152196C770E9CFDF91CF91C9
:102B50001F9108954091C0015091C1016091C2013F
:102B60007091C3018091C4019091C5010C947915B5
:102B70008091C50182958F7009F054C08091C20187
:102B8000882309F44FC080918E01A0918F0160913C
:102B9000C0017091C1014091C3015091C401B6E0E0
:102BA0008A1709F43FC090E041155105C1F17F3FFC
:102BB00011F46F3FA1F1B89FF001B99FF00D1124FE
:102BC000E057FE4F218172132AC02081621327C073
:102BD0002281211124C0238134812417350710F468
:102BE00021503109241B350B2C323140C0F4209187
:102BF000C5012F7020612093C50126E0289FF001B8
:102C0000299FF00D1124EB56FE4F80818F7080615B
:102C1000808380EC91E00E9426120C948915019625
:102C20008770BECF0895CF92DF92EF92FF920F93FD
:102C30001F93CF93DF93CDB7DEB762970FB6F894AB
:102C4000DEBF0FBECDBF8C0185E0F801DE011D9611
:102C500001900D928A95E1F7D8014C9111965C9103
:102C6000119712966C9112971396CD90DC90149751
:102C70003091C0017091C1018091C3019091C40154
:102C8000009709F473C17F3F19F43F3F09F46EC107
:102C9000E090C201EE2009F4C5C02091C501C8161C
:102CA000D90650F0F601E81BF90BCF01FF24F3948D
:102CB0008C329140C8F009C0809590958C0D9D1D77
:102CC000FF24F3948C32914078F0F12C207F09F0AE
:102CD000C6C07C2DD98AC88A89890E946A1580EC71
:102CE00091E00E942612B1C0822F807F09F045C07A
:102CF000751313C0341311C061110FC02F70206100
:102D00002093C5010E94AA1580EC91E00E94261232
:102D10008091C501F80185832EC0CD2819F15F3F50
:102D200011F44F3FF9F0F62E61111CC080918E0115
:102D300020918F0136E0821709F45BC090E0389F44
:102D4000F001399FF00D1124E057FE4F71815713A8
:102D500006C07081471303C07281711103C00196D0
:102D60008770E9CFF62E662309F41DC18091C50155
:102D700081608093C501F12C16C1751309C034130D
:102D800007C0611105C08091C501F8018583C8C0E5
:102D90004D875E878D859E856A8B0E9444156A8962
:102DA0008823E1F16623D1F12091C501822F82951C
:102DB0008F7090E0029774F08091C0019091C101F2
:102DC00098878F831986DB86CA862C87CE01079663
:102DD0000E94261286E0F801A0ECB1E001900D926D
:102DE0008A95E1F70E94B8150E94AA15FF24F39472
:102DF000DAC04D875E878D859E850E942D1A292F0A
:102E000022952F7030E0223031050CF0BFC09F704A
:102E100009F0B9C0805E883008F4C5C0C8010E94BE
:102E20002612E4CFC816D90608F453C0F601E81BF1
:102E3000F90BCF018C32914008F453C0F12C7C2D5A
:102E4000D98AC88A89890E946A15E0ECF1E086E097
:102E5000DF011D928A95E9F70E94AA15A4C0751397
:102E600014C0341312C0611110C08091C501F80163
:102E70008583C8010E94261286E0E0ECF1E0DF01C4
:102E80001D928A95E9F7FE2C8EC04D875E878D8551
:102E90009E856A8B0E9444156A89882309F4BECFF7
:102EA000662309F4BBCF2091C501822F82958F70D4
:102EB00090E002970CF48ECF8091C0019091C101F7
:102EC0009A8389831B82DD82CC822E83CE01019678
:102ED0007FCF809590958C0D9D1D8C32914008F090
:102EE000ADCFF62E662309F499CF75132EC0341397
:102EF0002CC02091C50120FD1FC0822F82958F70AC
:102F0000D9F0D80115962C9315978F3049F08F5F23
:102F1000982F9295907F822F8F70892B15968C9386
:102F2000C8010E94261286E0F801A0ECB1E00190F1
:102F30000D928A95E1F790CF86E0F801A0ECB1E020
:102F400001900D928A95E1F72EC04D875E878D85A1
:102F50009E850E94441581113DCF8091C5018160FD
:102F60008093C501C8010E9426121DC0662309F482
:102F700055CF4D875E878D859E850E944415882399
:102F800009F44CCF27CF811145CF0DC02430310536
:102F90000CF044CF9F7009F43DCFD80115969C9159
:102FA000907F09F037CF8F2D62960FB6F894DEBF71
:102FB0000FBECDBFDF91CF911F910F91FF90EF908A
:102FC000DF90CF9008951F93CF93DF93CDB7DEB7F7
:102FD0002C970FB6F894DEBF0FBECDBF4F83588736
:102FE00069877A878B879C87CE0107960E94131684
:102FF000882369F08F8198852A853B85232BF1F101
:103000009F3F09F063C08F3F09F060C037C086E082
:10301000FE013796DE01119601900D928A95E1F737
:103020006F817885EA85FB85309741F17F3F11F408
:103030006F3F21F120918F0130E0C9010196877027
:10304000992740918E0150E08417950709F447C0F5
:1030500069837A83FD83EC8396E0929FD001939FEE
:10306000B00D1124A057BE4FFE01319601900D9274
:103070009A95E1F780938F010E94891516E080915F
:103080008E0190918F018917C1F1189FC001112401
:1030900080579E4F0E941316882379F1E0918E018C
:1030A0001E9FF0011124E057FE4F40815181628143
:1030B0007381848195810E94791580918E0190E0C1
:1030C00001968770992780938E01D9CF4F815885BB
:1030D00069857A858B859C850E947915CFCF0E9462
:1030E000401510928F0110928E01E0ECF1E086E025
:1030F000DF011D928A95E9F7C1CF2C960FB6F8949F
:10310000DEBF0FBECDBFDF91CF911F910895DF923B
:10311000EF92FF920F931F93CF93DF93FC01892BC4
:1031200009F48AC0E12CF12CDD24D394EF0121961F
:103130008491853709F461C058F4843708F04EC093
:10314000843008F06AC08130D1F0823071F174C0EF
:10315000883709F45DC050F4863709F455C08737C5
:1031600009F06AC08E2D0E94261B54C09CE7980F60
:10317000903708F061C08F770E94F01150C08F0126
:103180000E5F1F4FFE01849190E2980F983050F42B
:103190008770FD2D01C0FF0F8A95EAF78F2F0E94DF
:1031A0002C1B14C00E94461113C08F010E5F1F4FCD
:1031B000FE01C49180E28C0F883060F4C7708D2DC1
:1031C00001C0880FCA95EAF70E94321B0E945D1B5E
:1031D000E80125C08C2F0E94F011FACF9F012E5FCD
:1031E0003F4FFE01C491CC2369F08FE99FE0019726
:1031F000F1F700C00000C150F6CF9F012E5F3F4F96
:10320000FE01F490E9010BC00E94161BE82E07C0D6
:103210000E94291B0E945D1B02C00E9446118F2D37
:10322000882341F0EFE9FFE03197F1F700C000009B
:103230008150F6CFFE017ACFDF91CF911F910F9190
:10324000FF90EF90DF9008956093CA017093CB01D7
:103250008093CC019093CD010E94DD1B0C942E1520
:103260006093C6017093C7018093C8019093C90110
:103270000E94DE1B0C942E1508950C9424190F93B4
:103280001F930091CA011091CB012091CC01309184
:10329000CD01602B712B822B932B1F910F910C94DE
:1032A00024190F931F930091CA011091CB01209113
:1032B000CC013091CD0160237123822393231F9190
:1032C0000F910C9424190F931F930091CA01109130
:1032D000CB012091CC013091CD016027712782274D
:1032E00093271F910F910C94241960E070E0CB019B
:1032F0000C9430190F931F9341E050E060E070E0B0
:103300008A019B0104C0000F111F221F331F8A95E1
:10331000D2F7C901B8011F910F910C9430190F9386
:103320001F9341E050E060E070E004C0440F551F7F
:10333000661F771F8A95D2F78091C6019091C701C9
:10334000A091C801B091C9018A019B01082B192BDA
:103350002A2B3B2BC901B8011F910F910C943019F6
:103360000F931F9341E050E060E070E004C0440F11
:10337000551F661F771F8A95D2F740955095609527
:1033800070958091C6019091C701A091C801B0913C
:10339000C9018A019B01082319232A233B23C90160
:1033A000B8011F910F910C9430190F931F9341E0B6
:1033B00050E060E070E004C0440F551F661F771FA7
:1033C0008A95D2F78091C6019091C701A091C8015A
:1033D000B091C9018A019B01082719272A273B2799
:1033E000C901B8011F910F910C9430190F931F93CD
:1033F0000091C6011091C7012091C8013091C90107
:10340000602B712B822B932B1F910F910C943019F1
:103410000F931F930091C6011091C7012091C8011D
:103420003091C90160237123822393231F910F914F
:103430000C9430190F931F930091C6011091C7018E
:103440002091C8013091C9016027712782279327F5
:103450001F910F910C9430190895CF92DF92EF9243
:10346000FF920F931F93CF93DF938C01C090CA01FB
:10347000D090CB01E090CC01F090CD014091C601FD
:103480005091C7016091C8017091C901C42AD52A21
:10349000E62AF72ACFE1D0E0D701C6010C2E04C0FE
:1034A000B695A795979587950A94D2F780FF07C0A0
:1034B000B8018C2F0E94171D8130910531F421979E
:1034C00058F7B80180E00E94171DDF91CF911F913E
:1034D0000F91FF90EF90DF90CF90089590910A01A7
:1034E000992321F090910B01911109C020910C01B9
:1034F00030910D01F90132969FEF40E030C0982FD6
:103500009695969596959F30A0F4E0910C01F091D8
:103510000D01E90FF11D877021E030E0A90102C023
:10352000440F551F8A95E2F7CA019181892B818347
:1035300008959091E30190FF23C01F928F938DED2A
:1035400093E09F938F930E94D2060F900F900F905D
:103550000F9008959F3F39F04F5F4E3041F05191E9
:103560005813F8CF0DC05111F7CF942FF5CF9F3FCF
:1035700039F0F901E90FF11D97FDFA95828308955D
:10358000089590910A01992321F090910B019111D6
:1035900009C020910C0130910D01F9013296205F94
:1035A0003F4F30C0982F9695969596959F30A8F4EA
:1035B000E0910C01F0910D01E90FF11D877021E000
:1035C00030E0A90102C0440F551F8A95E2F7CA01F5
:1035D000809591818923818308959091E30190FFE3
:1035E00016C01F928F938FEB93E09F938F930E944F
:1035F000D2060F900F900F900F9008953196E2171A
:10360000F30729F090819813F9CF1082F7CF08952E
:1036100081E090E0E0910C01F0910D01E80FF91FBD
:103620001082019680319105A9F708958091E201F9
:1036300008959091E201892B8093E201089580958D
:103640009091E20189238093E20108958093E20141
:1036500008951092E20108959091E101892B8093E1
:10366000E101089580959091E10189238093E10122
:1036700008951092E10108958093D0010E94531C97
:103680009093CF018093CE0108951092D0011092B3
:10369000CF011092CE01089580910C0190910D01FF
:1036A000FC0131969C01205F3F4F80E09191911188
:1036B0008F5FE217F307D1F70895E0910C01F091C5
:1036C0000D018091E2018083E0910C01F0910D01E8
:1036D00090818091E101892B80838091D0018823A2
:1036E000D9F10E94531C2091CE013091CF01821755
:1036F000930748F00E94531C2091CE013091CF01D6
:10370000821B930B0AC00E94531C2091CE01309162
:10371000CF0120953095820F931F8C32914070F02D
:103720008091E30180FF08C08BEF93E09F938F931C
:103730000E94D2060F900F900E94451BE0910C0151
:10374000F0910D0190818091D001892B80830E949E
:103750004C1B81110E94451B80910C0190910D0121
:103760000C94BE0F9093390180933801089582958F
:10377000982F9C7C392F36953695282F237344E05B
:10378000249FC0011124932F982B292F2A7A269544
:10379000892F8575880F822B08950895CF93DF9325
:1037A00000D000D01F92CDB7DEB70F900F900F90D2
:1037B0000F900F90DF91CF910895089508950C9484
:1037C000041108958091F801843021F11092E401F0
:1037D00020E488E190E00FB6F894A895809360000B
:1037E0000FBE2093600083B7817F846083BF83B75F
:1037F000816083BF7894889583B78E7F83BF0FB62F
:10380000F894A89580916000886180936000109280
:1038100060000FBE0895CF930E9412080E94040713
:103820000E941308C0E08C2F0E94DD07811104C0A4
:10383000CF5FC031C1F701C081E0CF9108950C94F2
:1038400040151F920F920FB60F9211248F939F93E2
:10385000AF93BF938091E401811113C08091E50182
:103860009091E601A091E701B091E8014196A11D78
:10387000B11D8093E5019093E601A093E701B09319
:10388000E801BF91AF919F918F910F900FBE0F9064
:103890001F90189582E084BD93E095BD9AEF97BD87
:1038A00080936E0008952FB7F8948091E501909170
:1038B000E601A091E701B091E8012FBF08952FB76D
:1038C000F8946091E5017091E6018091E701909193
:1038D000E8012FBF0895CF92DF92EF92FF920F93EE
:1038E0001F932FB7F8944091E5015091E601609144
:1038F000E7017091E8012FBF6A017B01EE24FF24EC
:103900008C0120E030E0C016D106E206F30610F488
:10391000415051099A01281B390BC9011F910F9180
:10392000FF90EF90DF90CF900895CF92DF92EF92CB
:10393000FF920F931F932FB7F894C090E501D0909A
:10394000E601E090E701F090E8012FBF97018601C2
:10395000061B170B280B390BC616D706E806F90607
:1039600018F0C901B80106C0C901B8016150710958
:10397000810991091F910F91FF90EF90DF90CF90F7
:1039800008951F920F920FB60F9211248F939F9359
:10399000AF93BF938091E5019091E601A091E7017B
:1039A000B091E8010196A11DB11D8093E5019093AE
:1039B000E601A093E701B093E801BF91AF919F9119
:1039C0008F910F900FBE0F901F9018950E94F90CC9
:1039D000F8942FEF87EA91E6215080409040E1F77C
:1039E00000C0000087E090EBDC018093020290931E
:1039F0000302A0930402B09305029CE088E10FB695
:103A0000F894A895809360000FBE90936000FFCF5C
:103A100028E0929FF0011124E80FF11DE052FF4FC2
:103A20008491982F90778F7092959F700895CF937F
:103A3000C82FCB010E94081D292F30E0E82FF0E0AD
:103A4000A90164E0440F551F6A95E1F74E2B5F2BE7
:103A50004038510519F480E090E012C088E0C89F1A
:103A6000200D311D112484E0220F331F8A95E1F7C8
:103A7000E20FF31FEE0FFF1FE050F849859194917C
:103A8000CF91089580E090E008950895CF92DF925D
:103A9000EF92FF920F931F93CF936C01C0E08C2F96
:103AA0000E94DD0700E010E0E82EF12CC701002E97
:103AB00002C0959587950A94E2F780FF16C0602FA3
:103AC0007C2F80E00E94171D9C018C159D0559F0EC
:103AD000832F807E932F907C11F0803A31F430E078
:103AE0002C153D0511F481E009C00F5F1F4F083010
:103AF0001105E1F6CF5FC03191F680E0CF911F91C3
:103B00000F91FF90EF90DF90CF900895CF93DF93C8
:103B1000EC018CE290E00E94461D882329F0CE0142
:103B2000DF91CF910C94461D80E0DF91CF910895F5
:103B3000CF930E94001F811102C00E94E61E84E103
:103B400094E00E943906C5E6C15049F00E9404077E
:103B50008FE39CE90197F1F700C00000F5CF8DE0FD
:103B600094E00E94390689E290E00E94861D81114E
:103B70002BC18AE290E00E94861D81110E94E61E00
:103B800085E090E00E94861D81110E94E61C0E9443
:103B9000E11B0E940B1F8093E30187E090E00E94ED
:103BA000861D8823C1F18BE190E00E94861D882349
:103BB00051F08091E30181FB222720F991E09227C7
:103BC00090FB81F90FC08EE090E00E94861D882353
:103BD00061F08091E30182FB222720F991E0922796
:103BE00090FB82F98093E30116C080E190E00E948F
:103BF000861D9091E301882341F093FB222720F951
:103C000081E0822780FB93F904C0892F809580FB97
:103C100090F99093E3018091E3010E940F1F0E94AD
:103C20001D1F8093010280EE90E00E94861D882374
:103C300041F080910102982F909590FB80F980933C
:103C4000010289E390E00E94861D882359F080914B
:103C5000010281FB222720F991E0922790FB81F954
:103C60008093010282EE90E00E94861D882359F025
:103C70008091010282FB222720F991E0922790FB9C
:103C800082F98093010286EE90E00E94861D8823CF
:103C900059F08091010283FB222720F991E09227BD
:103CA00090FB83F98093010283EE90E00E94861DD1
:103CB000882359F08091010284FB222720F991E0AA
:103CC000922790FB84F98093010285E390E00E94A3
:103CD000861D882359F08091010285FB222720F957
:103CE00091E0922790FB85F98093010281E390E0B7
:103CF0000E94861D882359F08091010286FB2227AD
:103D000020F991E0922790FB86F98093010281E1EE
:103D100090E00E94861D882359F08091010287FB64
:103D2000222720F991E0922790FB87F980930102E6
:103D3000809101020E94211F8091010287FB882748
:103D400080F980930B0187E290E00E94861DC82FC6
:103D50008EE190E00E94861D8111C2608FE190E0AB
:103D60000E94861D8111C46080E290E00E94861D41
:103D70008111C86081E290E00E94861D8111C061BE
:103D800082E290E00E94861D8111C06283E290E091
:103D90000E94861D8111C06484E290E00E94861D0D
:103DA000882311F0C06802C0CC2329F08C2F0E9418
:103DB000181F6C2F03C00E94141F682F70E080E052
:103DC00090E0CF910C943D19CF9108956DEE7EEF68
:103DD00080E090E00E947E2860E082E090E00E9417
:103DE000702860E083E090E00E94702860E084E04A
:103DF00090E00E94702860E085E090E00C947028CC
:103E000080E090E00E946A2821E08D3E9E4F09F0FC
:103E100020E0822F089582E090E00C946228682FC1
:103E200082E090E00C94702883E090E00C9462288B
:103E3000682F83E090E00C94702884E090E00C946C
:103E40006228682F84E090E00C9470288091EB0148
:103E500080FF0BC06091110185E0689FB0011124C3
:103E600075956795759567952BC081FF09C0609121
:103E7000110185E0689FB00111247595679520C0F8
:103E800082FF07C06091110185E0689FB001112495
:103E900017C09091EC019923D1F060911001961711
:103EA00088F72091110185E0289F90011124929FAD
:103EB000A001939F500D112470E0CA010E94342884
:103EC0006038710540F46115710539F002C065E094
:103ED00070E0862F08958FE7089581E0089580911E
:103EE000EB0180FF08C060910F0170E07595679548
:103EF0007595679521C081FF06C060910F0170E044
:103F00007595679519C082FF04C060910F0170E03C
:103F100010C09091EC019923C1F060910E019617A9
:103F2000A0F780910F01899FC001112470E00E94C9
:103F300034286038710528F46115710521F0862F49
:103F400008958FE7089581E0089561E070E0F4CF6F
:103F5000803F21F40E94261F819504C0813F29F4EF
:103F60000E94261F8093EF010895823F21F40E9452
:103F7000261F819504C0833F29F40E94261F809349
:103F8000EE010895893F19F40E946F1F05C08A3F12
:103F900031F40E946F1F81958093F00108958B3F4B
:103FA00021F40E946F1F819504C08C3F29F40E9468
:103FB0006F1F8093F1010895843F21F48091ED01FA
:103FC000816017C0853F21F48091ED01826011C0AE
:103FD000863F21F48091ED0184600BC0873F21F47E
:103FE0008091ED01886005C0883F31F48091ED013A
:103FF00080618093ED0108958D3F21F48091EB0164
:1040000081600BC08E3F21F48091EB01826005C07E
:104010008F3F29F48091EB0184608093EB01089538
:10402000803F39F48091EF0187FF6CC01092EF015F
:1040300069C0813F29F48091EF011816BCF362C07A
:104040009091EE01823F29F497FF5CC01092EE013F
:1040500059C0833F19F41916CCF354C0893F41F479
:104060008091F00118160CF04DC01092F0014AC07A
:104070008A3F29F48091F00187FF44C0F6CF8B3F3F
:1040800039F48091F10187FF3DC01092F1013AC0EF
:104090008C3F29F48091F1011816BCF333C0843FA2
:1040A00021F48091ED018E7F17C0853F21F480912E
:1040B000ED018D7F11C0863F21F48091ED018B7F52
:1040C0000BC0873F21F48091ED01877F05C0883FB9
:1040D00031F48091ED018F7E8093ED0113C08D3F0F
:1040E00021F48091EB018E7F0BC08E3F21F48091F3
:1040F000EB018D7F05C08F3F29F48091EB018B7F11
:104100008093EB018091EE0181110EC08091EF014F
:1041100081110AC08091F001811106C08091F101E6
:10412000811102C01092EC0108958091E30183FF98
:104130007EC080E594E00E9439068091ED011F92D7
:104140008F938BE494E09F938F930E94D20689E42F
:1041500094E00E9439068091EE01282F082E000C71
:10416000330B3F938F9386E494E09F938F930E9449
:10417000D20684E494E00E9439068091EF01282F52
:10418000082E000C330B3F938F9381E494E09F93B0
:104190008F930E94D2068FE394E00E9439068091AB
:1041A000F001282F082E000C330B3F938F938CE3E4
:1041B00094E09F938F930E94D2068AE394E00E943A
:1041C00039068091F101282F082E000C330B3F9304
:1041D0008F9387E394E09F938F930E94D20684E3AA
:1041E00094E00E9439068091EC011F928F9381E345
:1041F00094E09F938F930E94D2068FE294E00E94F6
:1042000039068091EB011F928F938CE294E09F938B
:104210008F930E94D20689E294E00E9439068DB7FE
:104220009EB74C960FB6F8949EBF0FBE8DBF8DEE15
:1042300091E00E9407100E94531C9093EA01809322
:10424000E90108951F93CF93DF938091E901909145
:10425000EA010E946B1CAC019091EC01992321F0C2
:104260002091120130E006C0209113018AE0289FBE
:10427000900111244217530708F485C08091EE0184
:10428000C091EF01D091F0011091F101811107C0AF
:10429000C11175C0D11173C0111171C074C09F3F9D
:1042A00019F09F5F9093EC01181624F40E94261FCA
:1042B0008093EE018091EE0187FF05C00E94261FCA
:1042C00081958093EE011C1624F40E94261F809392
:1042D000EF018091EF0187FF05C00E94261F8195A5
:1042E0008093EF016091EE01662331F1C091EF01FF
:1042F000CC2311F1062E000C770B880B990B0E9432
:104300002F2723E333E343E35FE30E9493270E94D5
:10431000F7266093EE016C2FCC0F770B880B990B6F
:104320000E942F2723E333E343E35FE30E949327B5
:104330000E94F7266093EF011D1624F40E946F1F60
:104340008093F0018091F00187FF05C00E946F1FEC
:1043500081958093F001111624F40E946F1F8093C1
:10436000F1018091F10187FF05C00E946F1F8195C7
:104370008093F101DF91CF911F910C9495209F3F85
:1043800009F08FCF97CFDF91CF911F910895EDEE78
:10439000F1E085E0DF011D928A95E9F71092EC01CA
:1043A0001092EB01089583E796E00E9439061F9270
:1043B00081E08F931F9285E08F9385E296E09F9333
:1043C0008F930E94D2060F900F900F900F900F9036
:1043D0000F9008958330E9F128F4813061F0823044
:1043E00009F10895853009F462C008F449C08630A7
:1043F00009F474C0089580911301262F30E0280F2E
:10440000311D2F3F310524F4680F6093130103C061
:104410008FEF80931301809113011F928F938EE58C
:1044200095E072C080911201262F30E0280F311DD7
:104430002F3F310524F4680F6093120103C08FEF02
:1044400080931201809112011F928F938CE495E06A
:104450005BC080911101262F30E0280F311D2F3FC6
:10446000310524F4680F6093110103C08FEF80932E
:104470001101809111011F928F9389E395E044C04F
:1044800080911001262F30E0280F311D2F3F31057C
:1044900024F4680F6093100103C08FEF8093100124
:1044A000809110011F928F9384E295E02DC080913E
:1044B0000F01262F30E0280F311D2F3F310524F446
:1044C000680F60930F0103C08FEF80930F018091FD
:1044D0000F011F928F938BE095E016C080910E0123
:1044E000262F30E0280F311D2F3F310524F4680FAF
:1044F00060930E0103C08FEF80930E0180910E0137
:104500001F928F9380EF94E09F938F930E94D20627
:104510000F900F900F900F900895833081F128F441
:10452000813059F08230D1F00895853009F449C0C6
:10453000B8F1863009F456C00895809113016817C8
:1045400020F4861B8093130102C010921301809106
:1045500013011F928F9381EE94E054C08091120159
:10456000681720F4861B8093120102C0109212017A
:10457000809112011F928F938FEC94E043C0809141
:104580001101681720F4861B8093110102C010925C
:104590001101809111011F928F938CEB94E032C036
:1045A00080911001681720F4861B8093100102C0CF
:1045B00010921001809110011F928F9387EA94E06E
:1045C00021C080910F01681720F4861B80930F0192
:1045D00002C010920F0180910F011F928F938EE8FD
:1045E00094E010C080910E01681720F4861B809320
:1045F0000E0102C010920E0180910E011F928F9346
:1046000083E794E09F938F930E94D2060F900F90C0
:104610000F900F900895CF93C82F1F928F9388E724
:1046200097E09F938F930E94D20681E090E0A0E0F4
:10463000B0E0BC01CD0104C0660F771F881F991F31
:10464000CA95D2F70E943D190F900F900F900F90CE
:10465000CF910C944015CF938B3109F4CBC108F066
:1046600049C08E3009F4DAC100F5873009F4A9C1D8
:10467000A8F4863009F05AC28091E301817F8E7FD1
:104680008093E3018DE797E00E94390688EB9BE079
:104690000E94390681E08093F30191C1883009F4CA
:1046A0005BC08B3009F487C141C2813109F426C255
:1046B00020F4803109F4C6C139C2863109F4DDC164
:1046C000893109F033C28CE29BE00E9439068FEFFA
:1046D0009AE00E94390688EC9AE00E94390681EA45
:1046E0009AE00E9439068DE49AE00E9439068FE133
:1046F0009AE063C1853309F413C268F4873209F480
:104700000FC228F48E3108F411C28D510CC28932C7
:1047100009F406C20BC2833438F48A3308F002C2AB
:10472000883309F448C102C2833409F4F9C18834DA
:1047300009F0FCC10E94401587EA9BE00E943906FF
:104740009FEF23ED80E3915020408040E1F700C0CF
:1047500000000E94E61C33C18CEB9BE00E943906EE
:104760008CE799E00E9439060E94141F1F928F93D4
:1047700089E799E09F938F930E94D20687E799E09B
:104780000E9439060E940B1FC82F84E699E00E9400
:1047900039061F92CF938FE599E09F938F930E94E4
:1047A000D2068DE599E00E94390683E599E00E94E2
:1047B00039068C2F81701F928F9380E599E09F932B
:1047C0008F930E94D2068EE499E00E94390684E419
:1047D00099E00E943906C1FB882780F91F928F93C8
:1047E00081E499E09F938F930E94D2068FE399E032
:1047F0000E94390683E399E00E943906C2FB8827AC
:1048000080F91F928F9380E399E09F938F930E948A
:10481000D2068EE299E00E94390685E299E00E9474
:104820003906C3FBCC27C0F91F92CF9382E299E0EF
:104830009F938F930E94D20680E299E00E943906EE
:104840000E941D1FC82F8CE099E00E9439061F921C
:10485000CF9387E099E09F938F930E94D20685E0E3
:1048600099E00E9439068CEE98E00E9439068C2F60
:1048700081701F928F9389EE98E09F938F930E948F
:10488000D2068DB79EB780960FB6F8949EBF0FBE26
:104890008DBF87EE98E00E94390680ED98E00E9477
:1048A0003906C1FB882780F91F928F938DEC98E021
:1048B0009F938F930E94D2068BEC98E00E9439065A
:1048C00089EB98E00E943906C2FB882780F91F9285
:1048D0008F9386EB98E09F938F930E94D20684EB90
:1048E00098E00E94390682EA98E00E943906C3FBEC
:1048F000882780F91F928F938FE998E09F938F9379
:104900000E94D2068DE998E00E94390683E998E07A
:104910000E943906C4FB882780F91F928F9380E993
:1049200098E09F938F930E94D2068EE898E00E94B1
:1049300039068CE798E00E943906C5FB882780F984
:104940001F928F9389E798E09F938F930E94D206DE
:1049500087E798E00E9439068BE598E00E943906C7
:10496000C6FB882780F91F928F9388E598E09F9374
:104970008F930E94D20686E598E00E9439068EE465
:1049800098E00E943906C7FBCC27C0F91F92CF934D
:104990008BE498E09F938F930E94D20689E498E07D
:1049A0000E9439068DB79EB74C960FB6F8949EBFFD
:1049B0000FBE8DBF04C084EA97E00E943906C1E0B3
:1049C000BAC08091E301C82FC17080FF09C08AE995
:1049D0009BE00E9439068091E301817F8E7F47C072
:1049E0008EE89BE00E9439068091E301816080930C
:1049F000E301E5CF9091E30191FBCC27C0F981E081
:104A0000C827892FC0FB81F98093E301CC2319F0DB
:104A100081E89BE027C083E79BE0CFCF9091E30143
:104A200092FBCC27C0F981E0C827892FC0FB82F90F
:104A30008093E301CC2319F084E69BE013C084E566
:104A40009BE0BBCF9091E30193FBCC27C0F981E0C1
:104A5000C827892FC0FB83F98093E301CC2351F051
:104A600088E49BE00E9439068091E3018160809395
:104A7000E30161C08BE39BE0A0CF81E19AE00E945B
:104A800039060E94B20F1F928F9387EF99E09F9390
:104A90008F930E94D20680910A011F928F9380EE1D
:104AA00099E09F938F930E94D206809176011F9286
:104AB0008F938DEC99E09F938F930E94D206809103
:104AC0000B011F928F938AEB99E09F938F930E9423
:104AD000D2060E945F1C9F938F937F936F9383EA0C
:104AE00099E09F938F930E94D2068DB79EB746960A
:104AF0000FB6F8949EBF0FBE8DBF61CF0E944015C8
:104B0000C0910B0181E0C827C0930B01CC2329F091
:104B100089E999E00E9439060EC08EE899E04DCFF0
:104B200080E001C089530E940B2349CF8CE899E0B3
:104B30000E943906C0E08C2FCF91089580E008953F
:104B400080E00895CF93C82F8091F301813071F0F8
:104B500020F0823009F44BC042C1E0910C01F09189
:104B60000D018081823209F03CC107C0E0910C0147
:104B7000F0910D018081823261F48C2F0E949E257C
:104B8000811104C08C2F0E942B232FC081E090E064
:104B90002CC08C2F0E94A025811126C0C431E1F0C9
:104BA00070F4CB3081F0C031D1F40E94D32180E782
:104BB00097E00E94390682E08093F30115C0C93264
:104BC00059F0C83361F48DE797E00E94390684E715
:104BD00097E00E94390608C01092F30104C18EE6E6
:104BE00097E00E943906FFC081E08170FEC0C432A8
:104BF00028F5CE3108F0C1C0CB30A1F1D0F4C730D8
:104C000009F0D3C08EE18093130182E380931201F7
:104C10008AE08093110184E18093100188E0809301
:104C20000F0188E280930E0184E196E00E9439062C
:104C3000BFC0C33149F1C431C1F0B7C0CB3409F4AE
:104C4000A9C028F4C93289F0C83361F0AEC0C135BB
:104C500009F49EC0C23509F499C0CE3409F0A5C04C
:104C60006AE09EC00E94D321A3C08091F2018823F4
:104C700019F01092F2019CC081E296E00E94390680
:104C800081E08093F301B1C08BEF95E00E9439067B
:104C900089EE95E00E943906809113011F928F934F
:104CA00086EE95E09F938F930E94D20684EE95E066
:104CB0000E94390682ED95E00E943906809112012A
:104CC0001F928F938FEC95E09F938F930E94D20653
:104CD0008DEC95E00E9439068EEB95E00E94390636
:104CE000809111011F928F938BEB95E09F938F938F
:104CF0000E94D20689EB95E00E94390688EA95E089
:104D00000E943906809110011F928F9385EA95E0E9
:104D10009F938F930E94D20683EA95E00E94390602
:104D20008EE895E00E94390680910F011F928F93C3
:104D30008BE895E09F938F930E94D20689E895E0D7
:104D40000E94390682E795E00E94390680910E01A3
:104D50001F928F938FE695E09F938F930E94D206C8
:104D60008DE695E00E9439068DB79EB748960FB63E
:104D7000F8949EBF0FBE8DBF1BC0CE51EC2FF0E04C
:104D8000E35DFE4F80818093F20112C061E003C0B9
:104D900061E006C06AE08091F2010E94EA2108C049
:104DA0008091F2010E948D2203C082E196E013C03F
:104DB0008091F201882369F01F928F938CE096E036
:104DC0009F938F930E94D2060F900F900F900F9099
:104DD00004C089E096E00E94390681E006C0109286
:104DE000F30180E002C080E000CFCF9108950E94DF
:104DF000FE266894B1110C948D2708950E947227A5
:104E000088F09F5798F0B92F9927B751B0F0E1F08B
:104E1000660F771F881F991F1AF0BA95C9F714C03B
:104E2000B13091F00E948C27B1E008950C948C274A
:104E3000672F782F8827B85F39F0B93FCCF3869574
:104E400077956795B395D9F73EF4909580957095D1
:104E500061957F4F8F4F9F4F0895E89409C097FB4E
:104E60003EF490958095709561957F4F8F4F9F4F41
:104E70009923A9F0F92F96E9BB279395F695879585
:104E800077956795B795F111F8CFFAF4BB0F11F448
:104E900060FF1BC06F5F7F4F8F4F9F4F16C08823EF
:104EA00011F096E911C0772321F09EE8872F762F25
:104EB00005C0662371F096E8862F70E060E02AF066
:104EC0009A95660F771F881FDAF7880F9695879552
:104ED00097F9089557FD9058440F551F59F05F3FBB
:104EE00071F04795880F97FB991F61F09F3F79F00C
:104EF00087950895121613061406551FF2CF46958E
:104F0000F1DF08C0161617061806991FF1CF86950F
:104F10007105610508940895E894BB2766277727F3
:104F2000CB0197F908950E94A6270C9417280E9498
:104F3000092838F00E94102820F0952311F00C94D5
:104F400000280C94062811240C948D270E946A27AF
:104F500070F3959FC1F3950F50E0551F629FF001CC
:104F6000729FBB27F00DB11D639FAA27F00DB11DE5
:104F7000AA1F649F6627B00DA11D661F829F22276E
:104F8000B00DA11D621F739FB00DA11D621F839FF5
:104F9000A00D611D221F749F3327A00D611D231FCB
:104FA000849F600D211D822F762F6A2F11249F5719
:104FB00050409AF0F1F088234AF0EE0FFF1FBB1F1C
:104FC000661F771F881F91505040A9F79E3F5105DB
:104FD00080F00C9400280C948D275F3FE4F3983EFA
:104FE000D4F3869577956795B795F795E7959F5F85
:104FF000C1F7FE2B880F911D9695879597F9089517
:1050000097F99F6780E870E060E008959FEF80EC7B
:10501000089500240A94161617061806090608951E
:1050200000240A9412161306140605060895092E84
:105030000394000C11F4882352F0BB0F40F4BF2BF3
:1050400011F460FF04C06F5F7F4F8F4F9F4F089533
:10505000991B79E004C0991F961708F0961B881FCA
:105060007A95C9F78095089597FB072E16F400945A
:1050700007D077FD09D00E944E2807FC05D03EF4EA
:10508000909581959F4F0895709561957F4F0895F4
:10509000EE0FFF1F0590F491E02D0994AA1BBB1B96
:1050A00051E107C0AA1FBB1FA617B70710F0A61B28
:1050B000B70B881F991F5A95A9F780959095BC0149
:1050C000CD010895F999FECF92BD81BDF89A992737
:1050D00080B50895A8E1B0E042E050E00C94852846
:1050E000262FF999FECF1FBA92BD81BD20BD0FB604
:1050F000F894FA9AF99A0FBE019608950E947028C2
:10510000272F0C947128DC01CB01FC01F999FECF0B
:1051100006C0F2BDE1BDF89A319600B40D9241503F
:0A5120005040B8F70895F894FFCF4F
:10512A001B080C09E908B50881080101D101280802
:10513A00140A321E404D3622395A030D03D702B5DE
:10514A00027C02EF01080221023A025A020102031A
:08515A00040506070809000026
:1068000088000000000000000400050006000700EA
:10681000080009000A000B000C000D000E000F001C
:1068200010001100120013001400150016001700CC
:10683000180019001A001B001C001D001E001F007C
:10684000200021002200230024002500260027002C
:10685000280035002A002B002C002D002E002F00D0
:106860003000310032003300340029003600370098
:106870003800E00000000000000000000000000000
:106880000000000000000000000000000000000008
:1068900000000000000000000000000000004F00A9
:1068A00050005100520000000000000000000000F5
:1068B00000000000000000000000000000000000D8
:1068C00000000000000000000000000000000000C8
:1068D00000000000000000000000000000000000B8
:1068E0000000000000000000890087008A008B0083
:1068F000F1A1E100E200E300F1A1E500E600000003
:106900000100010001000100EA4401000100E2442D
:106910000100010001005500460054004A004B00F0
:10692000560057004700480001000100E9440100FB
:106930000100010001000100010001003A003B00DC
:106940003C003D003E003F0040004100420043004B
:10695000580001004C00390001004400450052007D
:1069600001000100010050004F0081404D004E0029
:1069700051000100010001000100010001000100BF
:1069800001000100010001000100010001000100FF
:1069900001000100010001000100010001004D00A3
:1069A0004A004E004B0001000100010001000100FF
:1069B00001000100010001000100010001000100CF
:1069C00001000100010001000100010001000100BF
:1069D00001000100010001000100010001000100AF
:1069E0000100010001000100490001000100010057
:1069F000010001000100010001000100010001008F
:00000001FF
